:020000040000FA
:10000000000000000000000000008316FF239000A5
:100010000B308500831207309900A501702802304B
:10002000A900AA0B1128A90B1128A20B0F28003434
:1000300000001A28A60B1828A70B182800348207DE
:10004000000064348E34323464348E343234DC3420
:100050007E343234C8348E343234F034693432343D
:10006000F0347134F03461348E34143461348E34AD
:100070001434DC347E341434C8348E341434F03404
:100080005E341434F0346934F03461348E34143412
:1000900061348E341434F03447340134F03447344E
:1000A0001434F03454341434F03469341434F034E7
:1000B00071341434DC347E34F034F034503402348F
:1000C000F03450340234F03454340234F0346934AF
:1000D0000234F0345E340234F03469340234FF34D4
:1000E00018201820A50A25081F20A300FF3023068A
:1000F00003190528A50A25081F20A4002408A1002B
:1001000005150512832884288528A10B8228240838
:10011000A100051105168C288D288E28A10B8B288F
:10012000A30B7E28A50A25081F20A2000511051291
:040130000F20722802
:02400E00D43F9D
:00000001FF
